Microsoft (R) Macro Assembler Version 5.10                  2/14/25 23:44:19
DEBDATA.SAL - PC DOS                                        Page     1-1


					   PAGE    60,132 ;
					   TITLE DEBDATA.SAL - PC DOS
				;======================= START OF SPECIFICATIONS =========================
				;
				; MODULE NAME: DEBDATA.SAL
				;
				; DESCRIPTIVE NAME: DATA SEGMENT VALUE DEFINITION
				;
				; FUNCTION: PROVIDES ALL DATA SEGMENT DEFINITIONS.
				;
				; ENTRY POINT: NA
				;
				; INPUT: ANY VALUE IN DATA SEGMENT
				;
				; EXIT NORMAL: NA
				;
				; EXIT ERROR: NA
				;
				; INTERNAL REFERENCES: NA
				;
				; EXTERNAL REFERENCES: NA
				;
				; NOTES: THIS MODULE IS TO BE PREPPED BY SALUT WITH THE "PR" OPTIONS.
				;	 LINK DEBUG+DEBCOM1+DEBCOM2+DEBCOM3+DEBASM+DEBUASM+DEBERR+
				;	      DEBCONST+DEBDATA+DEBMES
				;
				; REVISION HISTORY:
				;
				;	AN000	VERSION 4.00 - REVISIONS MADE RELATE TO THE FOLLOWING:
				;
				;				- IMPLEMENT DBCS HANDLING	DMS:6/17/87
				;				- IMPLEMENT MESSAGE RETRIEVER	DMS:6/17/87
				;				- > 32 MB SUPPORT		DMS:6/17/87
				;
				; COPYRIGHT: "MS DOS DEBUG UTILITY"
				;	     "VERSION 4.00 (C) COPYRIGHT 1988 Microsoft"
				;	     "LICENSED MATERIAL - PROPERTY OF Microsoft  "
				;
				;======================= END OF SPECIFICATIONS ===========================
				
				.LIST
				.CREF
 0000				CODE	   SEGMENT PUBLIC BYTE
 0000				CODE	   ENDS
				
 0000				CONST	   SEGMENT PUBLIC BYTE
 0000				CONST	   ENDS
				
 0000				DATA	   SEGMENT PUBLIC BYTE
 0000				DATA	   ENDS
				
 0000				CSTACK	   SEGMENT STACK
 0000				CSTACK	   ENDS
				
				DG	   GROUP CODE,CONST,CSTACK,DATA
				
 0000				DATA	   SEGMENT PUBLIC BYTE
					   PUBLIC PARITYFLAG,XNXOPT,XNXCMD,SWITCHAR,EXTPTR,HANDLE,TRANSADD
					   PUBLIC PARSERR,ASMADD,DISADD,DISCNT,ASMSP,INDEX,DEFDUMP,DEFLEN
					   PUBLIC REGSAVE,SEGSAVE,OFFSAVE,TEMP,BUFFER,BYTCNT,OPCODE,AWORD
					   PUBLIC REGMEM,MIDFLD,MODE,NSEG,BRKCNT,TCOUNT,ASSEM_CNT
					   PUBLIC ASSEM1,ASSEM2,ASSEM3,ASSEM4,ASSEM5,ASSEM6,BYTEBUF,BPTAB
					   PUBLIC DIFLG,SIFLG,BXFLG,BPFLG,NEGFLG,NUMFLG,MEMFLG,REGFLG
					   PUBLIC MOVFLG,TSTFLG,SEGFLG,LOWNUM,HINUM,F8087,DIRFLG,DATAEND
					   PUBLIC BEGSEG,CREATE_LONG,ARG_BUF_INDEX
					   PUBLIC FILEEND,FILESTRT,SSINTSAV,BPINTSAV
					   PUBLIC FZTRACE, PREV24, FIN24
				
					   public rel_read_write_tab		;an000;relative read/write
										;      table
					   public rel_low_sec			;an000;sector add. low word
					   public rel_high_sec			;an000;sector add. high word
					   public rel_sec_num			;an000;# of sectors to access
					   public rel_rw_add			;an000;transfer address
				
					   public lbtbl 			;an000;lead byte table pointer
Microsoft (R) Macro Assembler Version 5.10                  2/14/25 23:44:19
DEBDATA.SAL - PC DOS                                        Page     1-2
                                                            

				
					public xm_page				;an000;
					public xm_log				;an000;
					public xm_phy				;an000;
					public xm_handle			;an000;
					public xm_handle_ret			;an000;
					public xm_page_cnt			;an000;
					public xm_handle_pages_buf		;an000;
					public xm_frame 			;an000;
					public xm_deall_han			;an000;
					public xm_alloc_pg			;an000;
					public xm_total_pg			;an000;
					public xm_han_total			;an000;
					public xm_han_alloc			;an000;
				
				;=========================================================================
				; REL_READ_WRITE_TAB : This table provides the new generic IOCTL primitive
				;		       read/write with its values.
				;
				;	Date	  : 6/17/87
				;=========================================================================
				
 0000				REL_READ_WRITE_TAB	label	dword		;an000;relative read/write
										;      table
 0000  0000				rel_low_sec	dw	?		;an000;sector add. low word
 0002  0000				rel_high_sec	dw	?		;an000;sector add. high word
 0004  0000				rel_sec_num	dw	?		;an000;# of sectors to write
 0006  00000000				rel_rw_add	dd	?		;an000;holds the segment
										;      & offset of the
										;      transfer address
				
				;=========================================================================
				
 000A  00000000			lbtbl		dd	?			;an000;lead byte table pointer
				
 000E  00				xm_page        db   ?			;an000;page count to allocate
 000F  00				xm_log	       db   ?			;an000;log. page to map
 0010  00				xm_phy	       db   ?			;an000;phy. page to map
 0011  0000				xm_deall_han   dw   ?			;an000;handle to deallocate
 0013  0000				xm_handle      dw   ?			;an000;handle to map
 0015  0000				xm_handle_ret  dw   ?			;an000;handle created
				
				
 0017  0000				xm_page_cnt    dw   ?			;an000;current page count
				
 0019  0400[				xm_handle_pages_buf db	 1024 dup(0)	;an000;hold handle pages
	   00			
			 ]	
				
				
 0419  0000				xm_frame	dw  ?			;an000;holds frame segment
				
 041B  0000				xm_alloc_pg	dw  ?			;an000;active page count
				
 041D  0000				xm_total_pg	dw  ?			;an000;total possible page cnt.
				
 041F  0000				xm_han_total	dw  ?			;an000;total possible handles
				
 0421  0000				xm_han_alloc	dw  ?			;an000;handles allocated
				
					   IF	IBMVER
					       PUBLIC OLD_MASK
 0423  00			OLD_MASK       DB   ?
					   ENDIF
 0424  00000000			PREV24	   DD	?			; prevvious INT 24 handler
 0428  00			FIN24	   DB	0			; TRUE => in the process of cleaning up
 0429  00			FZTRACE    DB	0			; TRUE => in a Ztrace
 042A  0000			FILEEND    DW	?			; ARR 2.4
 042C  0000			FILESTRT   DW	?			; ARR 2.4
 042E  00000000			SSINTSAV   DD	?			; ARR 2.4
 0432  00000000			BPINTSAV   DD	?			; ARR 2.4
				
 0436  00			PARITYFLAG DB	0
				
				PUBLIC	   SAVESTATE
 0437  0000			SAVESTATE  DPL	<>			; storage for extended error info
Microsoft (R) Macro Assembler Version 5.10                  2/14/25 23:44:19
DEBDATA.SAL - PC DOS                                        Page     1-3
                                                            

 0439  0000			
 043B  0000			
 043D  0000			
 043F  0000			
 0441  0000			
 0443  0000			
 0445  0000			
 0447  0000			
 0449  0000			
 044B  0000			
				
				
 044D  00			XNXOPT	   DB	?			; AL OPTION FOR DOS COMMAND
 044E  00			XNXCMD	   DB	?			; DOS COMMAND FOR OPEN_A_FILE TO PERFORM
 044F  00			SWITCHAR   DB	?			; CURRENT SWITCH CHARACTER
 0450  0000			EXTPTR	   DW	?			; POINTER TO FILE EXTENSION
 0452  0000			HANDLE	   DW	?			; CURRENT HANDLE
 0454  00000000			TRANSADD   DD	?			; TRANSFER ADDRESS
				
 0458  00			PARSERR    DB	?
 0459  0004[			ASMADD	   DB	4 DUP (?)
	   ??			
			 ]	
				
 045D  0004[			DISADD	   DB	4 DUP (?)
	   ??			
			 ]	
				
 0461  0000			DISCNT	   DW	?
 0463  0000			ASMSP	   DW	?			; SP AT ENTRY TO ASM
 0465  0000			INDEX	   DW	?
 0467  0004[			DEFDUMP    DB	4 DUP (?)
	   ??			
			 ]	
				
 046B  0000			DEFLEN	   DW	?
 046D  0000			REGSAVE    DW	?
 046F  0000			SEGSAVE    DW	?
 0471  0000			OFFSAVE    DW	?
				
				;Do NOT move this dword variable - it sets up a long call for
				;a Create_process_data_block call issued in DEBUG
 0473				CREATE_LONG LABEL DWORD
 0473  0100				   DW	100H
 0475  0000			BEGSEG	   DW	?
				
				; The following data areas are destroyed during hex file read
 0477  0004[			TEMP	   DB	4 DUP(?)
	   ??			
			 ]	
				
 047B				BUFFER	   LABEL BYTE
 047B  00			BYTCNT	   DB	?
 047C  0000			ARG_BUF_INDEX DW ?
 047E  0000			OPCODE	   DW	?
 0480  00			AWORD	   DB	?
 0481  00			REGMEM	   DB	?
 0482  00			MIDFLD	   DB	?
 0483  00			MODE	   DB	?
 0484  0000			NSEG	   DW	?
 0486  0000			BRKCNT	   DW	?			; Number of breakpoints
 0488  0000			TCOUNT	   DW	?			; Number of steps to trace
 048A  00			ASSEM_CNT  DB	?			; preserve order of assem_cnt and assem1
 048B  00			ASSEM1	   DB	?
 048C  00			ASSEM2	   DB	?
 048D  00			ASSEM3	   DB	?
 048E  00			ASSEM4	   DB	?
 048F  00			ASSEM5	   DB	?
 0490  00			ASSEM6	   DB	?			; preserve order of assemx and bytebuf
 0491  0050[			BYTEBUF    DB	BUFLEN	DUP (?) 	; Table used by LIST
	   ??			
			 ]	
				
 04E1  0032[			BPTAB	   DB	BPLEN	DUP (?) 	; Breakpoint table
	   ??			
			 ]	
Microsoft (R) Macro Assembler Version 5.10                  2/14/25 23:44:19
DEBDATA.SAL - PC DOS                                        Page     1-4
                                                            

				
 0513  00			DIFLG	   DB	?
 0514  00			SIFLG	   DB	?
 0515  00			BXFLG	   DB	?
 0516  00			BPFLG	   DB	?
 0517  00			NEGFLG	   DB	?
 0518  00			NUMFLG	   DB	?			; ZERO MEANS NO NUMBER SEEN
 0519  00			MEMFLG	   DB	?
 051A  00			REGFLG	   DB	?
 051B  00			MOVFLG	   DB	?
 051C  00			TSTFLG	   DB	?
 051D  00			SEGFLG	   DB	?
 051E  0000			LOWNUM	   DW	?
 0520  0000			HINUM	   DW	?
 0522  00			F8087	   DB	?
 0523  00			DIRFLG	   DB	?
 0524  0157[				   DB	BUFFER+BUFSIZ-$ DUP (?)
	   ??			
			 ]	
				
				
 067B				DATAEND    LABEL WORD
				
 067B				DATA	   ENDS
					   END

Microsoft (R) Macro Assembler Version 5.10                  2/14/25 23:44:19
DEBDATA.SAL - PC DOS                                        Symbols-1


Macros:

		N a m e			Lines

ARGVAR . . . . . . . . . . . . .  	  23
ASMVAR . . . . . . . . . . . . .  	   3
ASMVARS  . . . . . . . . . . . .  	   3
ASSERT . . . . . . . . . . . . .  	   0
CALLINSTALL  . . . . . . . . . .  	  12
DOSASSUME  . . . . . . . . . . .  	   3
ENTER  . . . . . . . . . . . . .  	   3
ENTERCRIT  . . . . . . . . . . .  	   1
ERRNZ  . . . . . . . . . . . . .  	   4
FMT  . . . . . . . . . . . . . .  	   0
LEAVE  . . . . . . . . . . . . .  	   2
LEAVECRIT  . . . . . . . . . . .  	   1
LOCALVAR . . . . . . . . . . . .  	  23

Structures and Records:

                N a m e                 Width   # fields
                                        Shift   Width   Mask    Initial

ARENA  . . . . . . . . . . . . .  	0010	0005
  ARENA_SIGNATURE  . . . . . . .  	0000
  ARENA_OWNER  . . . . . . . . .  	0001
  ARENA_SIZE . . . . . . . . . .  	0003
  ARENA_RESERVED . . . . . . . .  	0005
  ARENA_NAME . . . . . . . . . .  	0008
A_BPB  . . . . . . . . . . . . .  	001F	000F
  BPB_BYTESPERSECTOR . . . . . .  	0000
  BPB_SECTORSPERCLUSTER  . . . .  	0002
  BPB_RESERVEDSECTORS  . . . . .  	0003
  BPB_NUMBEROFFATS . . . . . . .  	0005
  BPB_ROOTENTRIES  . . . . . . .  	0006
  BPB_TOTALSECTORS . . . . . . .  	0008
  BPB_MEDIADESCRIPTOR  . . . . .  	000A
  BPB_SECTORSPERFAT  . . . . . .  	000B
  BPB_SECTORSPERTRACK  . . . . .  	000D
  BPB_HEADS  . . . . . . . . . .  	000F
  BPB_HIDDENSECTORS  . . . . . .  	0011
  BPB_BIGTOTALSECTORS  . . . . .  	0015
BPBLOCK  . . . . . . . . . . . .  	000D	0008
  BPSECSZ  . . . . . . . . . . .  	0000
  BPCLUS . . . . . . . . . . . .  	0002
  BPRES  . . . . . . . . . . . .  	0003
  BPFTCNT  . . . . . . . . . . .  	0005
  BPDRCNT  . . . . . . . . . . .  	0006
  BPSCCNT  . . . . . . . . . . .  	0008
  BPMEDIA  . . . . . . . . . . .  	000A
  BPFTSEC  . . . . . . . . . . .  	000B
BUFFER_HASH_ENTRY  . . . . . . .  	0008	0004
  EMS_PAGE_NUM . . . . . . . . .  	0000
  BUFFER_BUCKET  . . . . . . . .  	0002
  DIRTY_COUNT  . . . . . . . . .  	0006
  BUFFER_RESERVED  . . . . . . .  	0007
BUFFINFO . . . . . . . . . . . .  	0023	000F
  HASH_PTR . . . . . . . . . . .  	0000
  HASH_COUNT . . . . . . . . . .  	0004
  CACHE_PTR  . . . . . . . . . .  	0006
  CACHE_COUNT  . . . . . . . . .  	000A
  EMS_SAFE_FLAG  . . . . . . . .  	000C
  EMS_LAST_PAGE  . . . . . . . .  	000D
  EMS_FIRST_PAGE . . . . . . . .  	0011
  EMS_NPA640 . . . . . . . . . .  	0015
  EMS_MODE . . . . . . . . . . .  	0017
  EMS_HANDLE . . . . . . . . . .  	0018
  EMS_PAGEFRAME_NUMBER . . . . .  	001A
  EMS_SEG_CNT  . . . . . . . . .  	001C
  EMS_PAGE_FRAME . . . . . . . .  	001E
  EMS_RESERVED . . . . . . . . .  	0020
  EMS_MAP_BUFF . . . . . . . . .  	0022
CURDIR_LIST  . . . . . . . . . .  	0058	000A
  CURDIR_TEXT  . . . . . . . . .  	0000
  CURDIR_FLAGS . . . . . . . . .  	0043
  CURDIR_DEVPTR  . . . . . . . .  	0045
Microsoft (R) Macro Assembler Version 5.10                  2/14/25 23:44:19
DEBDATA.SAL - PC DOS                                        Symbols-2


  CURDIR_ID  . . . . . . . . . .  	0049
  CURDIR_USER_WORD . . . . . . .  	004D
  CURDIR_END . . . . . . . . . .  	004F
  CURDIR_TYPE  . . . . . . . . .  	0051
  CURDIR_IFS_HDR . . . . . . . .  	0052
  CURDIR_FSDA  . . . . . . . . .  	0056
DIR_ENTRY  . . . . . . . . . . .  	0020	000B
  DIR_NAME . . . . . . . . . . .  	0000
  DIR_ATTR . . . . . . . . . . .  	000B
  DIR_CODEPG . . . . . . . . . .  	000C
  DIR_EXTCLUSTER . . . . . . . .  	000E
  DIR_ATTR2  . . . . . . . . . .  	0010
  DIR_PAD  . . . . . . . . . . .  	0011
  DIR_TIME . . . . . . . . . . .  	0016
  DIR_DATE . . . . . . . . . . .  	0018
  DIR_FIRST  . . . . . . . . . .  	001A
  DIR_SIZE_L . . . . . . . . . .  	001C
  DIR_SIZE_H . . . . . . . . . .  	001E
DPB  . . . . . . . . . . . . . .  	0021	0012
  DPB_DRIVE  . . . . . . . . . .  	0000
  DPB_UNIT . . . . . . . . . . .  	0001
  DPB_SECTOR_SIZE  . . . . . . .  	0002
  DPB_CLUSTER_MASK . . . . . . .  	0004
  DPB_CLUSTER_SHIFT  . . . . . .  	0005
  DPB_FIRST_FAT  . . . . . . . .  	0006
  DPB_FAT_COUNT  . . . . . . . .  	0008
  DPB_ROOT_ENTRIES . . . . . . .  	0009
  DPB_FIRST_SECTOR . . . . . . .  	000B
  DPB_MAX_CLUSTER  . . . . . . .  	000D
  DPB_FAT_SIZE . . . . . . . . .  	000F
  DPB_DIR_SECTOR . . . . . . . .  	0011
  DPB_DRIVER_ADDR  . . . . . . .  	0013
  DPB_MEDIA  . . . . . . . . . .  	0017
  DPB_FIRST_ACCESS . . . . . . .  	0018
  DPB_NEXT_DPB . . . . . . . . .  	0019
  DPB_NEXT_FREE  . . . . . . . .  	001D
  DPB_FREE_CNT . . . . . . . . .  	001F
DPL  . . . . . . . . . . . . . .  	0016	000B
  DPL_AX . . . . . . . . . . . .  	0000
  DPL_BX . . . . . . . . . . . .  	0002
  DPL_CX . . . . . . . . . . . .  	0004
  DPL_DX . . . . . . . . . . . .  	0006
  DPL_SI . . . . . . . . . . . .  	0008
  DPL_DI . . . . . . . . . . . .  	000A
  DPL_DS . . . . . . . . . . . .  	000C
  DPL_ES . . . . . . . . . . . .  	000E
  DPL_RESERVED . . . . . . . . .  	0010
  DPL_UID  . . . . . . . . . . .  	0012
  DPL_PID  . . . . . . . . . . .  	0014
EXEC0  . . . . . . . . . . . . .  	000E	0004
  EXEC0_ENVIRON  . . . . . . . .  	0000
  EXEC0_COM_LINE . . . . . . . .  	0002
  EXEC0_5C_FCB . . . . . . . . .  	0006
  EXEC0_6C_FCB . . . . . . . . .  	000A
EXEC1  . . . . . . . . . . . . .  	0016	0008
  EXEC1_ENVIRON  . . . . . . . .  	0000
  EXEC1_COM_LINE . . . . . . . .  	0002
  EXEC1_5C_FCB . . . . . . . . .  	0006
  EXEC1_6C_FCB . . . . . . . . .  	000A
  EXEC1_SP . . . . . . . . . . .  	000E
  EXEC1_SS . . . . . . . . . . .  	0010
  EXEC1_IP . . . . . . . . . . .  	0012
  EXEC1_CS . . . . . . . . . . .  	0014
EXEC3  . . . . . . . . . . . . .  	0004	0002
  EXEC3_LOAD_ADDR  . . . . . . .  	0000
  EXEC3_RELOC_FAC  . . . . . . .  	0002
EXE_FILE . . . . . . . . . . . .  	0020	000F
  EXE_SIGNATURE  . . . . . . . .  	0000
  EXE_LEN_MOD_512  . . . . . . .  	0002
  EXE_PAGES  . . . . . . . . . .  	0004
  EXE_RLE_COUNT  . . . . . . . .  	0006
  EXE_PAR_DIR  . . . . . . . . .  	0008
  EXE_MIN_BSS  . . . . . . . . .  	000A
  EXE_MAX_BSS  . . . . . . . . .  	000C
  EXE_SS . . . . . . . . . . . .  	000E
  EXE_SP . . . . . . . . . . . .  	0010
Microsoft (R) Macro Assembler Version 5.10                  2/14/25 23:44:19
DEBDATA.SAL - PC DOS                                        Symbols-3


  EXE_CHKSUM . . . . . . . . . .  	0012
  EXE_IP . . . . . . . . . . . .  	0014
  EXE_CS . . . . . . . . . . . .  	0016
  EXE_RLE_TABLE  . . . . . . . .  	0018
  EXE_IOV  . . . . . . . . . . .  	001A
  EXE_SYM_TAB  . . . . . . . . .  	001C
EXT_OPEN_PARM  . . . . . . . . .  	0006	0002
  EXT_SET_LIST . . . . . . . . .  	0000
  EXT_NUM_OF_PARM  . . . . . . .  	0004
FIND_BUF . . . . . . . . . . . .  	002B	000C
  FIND_BUF_DRIVE . . . . . . . .  	0000
  FIND_BUF_NAME  . . . . . . . .  	0001
  FIND_BUF_SATTR . . . . . . . .  	000C
  FIND_BUF_LASTENT . . . . . . .  	000D
  FIND_BUF_DIRSTART  . . . . . .  	000F
  FIND_BUF_NETID . . . . . . . .  	0011
  FIND_BUF_ATTR  . . . . . . . .  	0015
  FIND_BUF_TIME  . . . . . . . .  	0016
  FIND_BUF_DATE  . . . . . . . .  	0018
  FIND_BUF_SIZE_L  . . . . . . .  	001A
  FIND_BUF_SIZE_H  . . . . . . .  	001C
  FIND_BUF_PNAME . . . . . . . .  	001E
INTERNAT_BLOCK . . . . . . . . .  	0018	0015
  DATE_TIM_FORMAT  . . . . . . .  	0000
  CURRENCY_SYM . . . . . . . . .  	0002
  THOUS_SEP  . . . . . . . . . .  	0007
  DECIMAL_SEP  . . . . . . . . .  	0009
  DATE_SEP . . . . . . . . . . .  	000B
  TIME_SEP . . . . . . . . . . .  	000D
  BIT_FIELD  . . . . . . . . . .  	000F
  CURRENCY_CENTS . . . . . . . .  	0010
  TIME_24  . . . . . . . . . . .  	0011
  MAP_CALL . . . . . . . . . . .  	0012
  DATA_SEP . . . . . . . . . . .  	0016
PROCESS_DATA_BLOCK . . . . . . .  	005C	0011
  PDB_EXIT_CALL  . . . . . . . .  	0000
  PDB_BLOCK_LEN  . . . . . . . .  	0002
  PDB_CPM_CALL . . . . . . . . .  	0005
  PDB_EXIT . . . . . . . . . . .  	000A
  PDB_CTRL_C . . . . . . . . . .  	000E
  PDB_FATAL_ABORT  . . . . . . .  	0012
  PDB_PARENT_PID . . . . . . . .  	0016
  PDB_JFN_TABLE  . . . . . . . .  	0018
  PDB_ENVIRON  . . . . . . . . .  	002C
  PDB_USER_STACK . . . . . . . .  	002E
  PDB_JFN_LENGTH . . . . . . . .  	0032
  PDB_JFN_POINTER  . . . . . . .  	0034
  PDB_NEXT_PDB . . . . . . . . .  	0038
  PDB_PAD1 . . . . . . . . . . .  	003C
  PDB_CALL_SYSTEM  . . . . . . .  	0050
  PDB_PAD2 . . . . . . . . . . .  	0055
SF . . . . . . . . . . . . . . .  	0008	0003
  SFLINK . . . . . . . . . . . .  	0000
  SFCOUNT  . . . . . . . . . . .  	0004
  SFTABLE  . . . . . . . . . . .  	0006
SF_ENTRY . . . . . . . . . . . .  	003B	0014
  SF_REF_COUNT . . . . . . . . .  	0000
  SF_MODE  . . . . . . . . . . .  	0002
  SF_ATTR  . . . . . . . . . . .  	0004
  SF_FLAGS . . . . . . . . . . .  	0005
  SF_DEVPTR  . . . . . . . . . .  	0007
  SF_FIRCLUS . . . . . . . . . .  	000B
  SF_TIME  . . . . . . . . . . .  	000D
  SF_DATE  . . . . . . . . . . .  	000F
  SF_SIZE  . . . . . . . . . . .  	0011
  SF_POSITION  . . . . . . . . .  	0015
  SF_CLUSPOS . . . . . . . . . .  	0019
  SF_DIRSEC  . . . . . . . . . .  	001B
  SF_DIRPOS  . . . . . . . . . .  	001F
  SF_NAME  . . . . . . . . . . .  	0020
  SF_CHAIN . . . . . . . . . . .  	002B
  SF_UID . . . . . . . . . . . .  	002F
  SF_PID . . . . . . . . . . . .  	0031
  SF_MFT . . . . . . . . . . . .  	0033
  SF_LSTCLUS . . . . . . . . . .  	0035
  SF_IFS_HDR . . . . . . . . . .  	0037
Microsoft (R) Macro Assembler Version 5.10                  2/14/25 23:44:19
DEBDATA.SAL - PC DOS                                        Symbols-4


SYMBOL_ENTRY . . . . . . . . . .  	0106	0004
  SYM_VALUE  . . . . . . . . . .  	0000
  SYM_TYPE . . . . . . . . . . .  	0004
  SYM_LEN  . . . . . . . . . . .  	0006
  SYM_NAME . . . . . . . . . . .  	0007
SYSINITVARS  . . . . . . . . . .  	0047	0018
  SYSI_DPB . . . . . . . . . . .  	0000
  SYSI_SFT . . . . . . . . . . .  	0004
  SYSI_CLOCK . . . . . . . . . .  	0008
  SYSI_CON . . . . . . . . . . .  	000C
  SYSI_MAXSEC  . . . . . . . . .  	0010
  SYSI_BUF . . . . . . . . . . .  	0012
  SYSI_CDS . . . . . . . . . . .  	0016
  SYSI_FCB . . . . . . . . . . .  	001A
  SYSI_KEEP  . . . . . . . . . .  	001E
  SYSI_NUMIO . . . . . . . . . .  	0020
  SYSI_NCDS  . . . . . . . . . .  	0021
  SYSI_DEV . . . . . . . . . . .  	0022
  SYSI_ATTR  . . . . . . . . . .  	0026
  SYSI_STRAT . . . . . . . . . .  	0028
  SYSI_INTER . . . . . . . . . .  	002A
  SYSI_NAME  . . . . . . . . . .  	002C
  SYSI_SPLICE  . . . . . . . . .  	0034
  SYSI_IBMDOS_SIZE . . . . . . .  	0035
  SYSI_IFS_DOSCALL@  . . . . . .  	0037
  SYSI_IFS . . . . . . . . . . .  	003B
  SYSI_BUFFERS . . . . . . . . .  	003F
  SYSI_BOOT_DRIVE  . . . . . . .  	0043
  SYSI_DWMOVE  . . . . . . . . .  	0044
  SYSI_EXT_MEM . . . . . . . . .  	0045
SYSINITVARS_EXT  . . . . . . . .  	0008	0002
  SYSI_INITVARS  . . . . . . . .  	0000
  SYSI_COUNTRY_TAB . . . . . . .  	0004
SYS_FCB  . . . . . . . . . . . .  	0025	000C
  FCB_DRIVE  . . . . . . . . . .  	0000
  FCB_NAME . . . . . . . . . . .  	0001
  FCB_EXT  . . . . . . . . . . .  	0009
  FCB_EXTENT . . . . . . . . . .  	000C
  FCB_RECSIZ . . . . . . . . . .  	000E
  FCB_FILSIZ . . . . . . . . . .  	0010
  FCB_DRVBP  . . . . . . . . . .  	0012
  FCB_FDATE  . . . . . . . . . .  	0014
  FCB_FTIME  . . . . . . . . . .  	0016
  FCB_RESERVED . . . . . . . . .  	0018
  FCB_NR . . . . . . . . . . . .  	0020
  FCB_RR . . . . . . . . . . . .  	0021
USER_ENVIRON . . . . . . . . . .  	0018	000C
  USER_AX  . . . . . . . . . . .  	0000
  USER_BX  . . . . . . . . . . .  	0002
  USER_CX  . . . . . . . . . . .  	0004
  USER_DX  . . . . . . . . . . .  	0006
  USER_SI  . . . . . . . . . . .  	0008
  USER_DI  . . . . . . . . . . .  	000A
  USER_BP  . . . . . . . . . . .  	000C
  USER_DS  . . . . . . . . . . .  	000E
  USER_ES  . . . . . . . . . . .  	0010
  USER_IP  . . . . . . . . . . .  	0012
  USER_CS  . . . . . . . . . . .  	0014
  USER_F . . . . . . . . . . . .  	0016

Segments and Groups:

                N a m e         	Length	 Align	Combine Class

DG . . . . . . . . . . . . . . .  	GROUP
  CODE . . . . . . . . . . . . .  	0000	BYTE	PUBLIC	
  CONST  . . . . . . . . . . . .  	0000	BYTE	PUBLIC	
  CSTACK . . . . . . . . . . . .  	0000	PARA	STACK	
  DATA . . . . . . . . . . . . .  	067B	BYTE	PUBLIC	
Microsoft (R) Macro Assembler Version 5.10                  2/14/25 23:44:19
DEBDATA.SAL - PC DOS                                        Symbols-5


Symbols:            

                N a m e         	Type	 Value	 Attr

ABORT  . . . . . . . . . . . . .  	NUMBER	0000	
ACCESS_MASK  . . . . . . . . . .  	NUMBER	000F	
ACTION_CREATED_OPENED  . . . . .  	NUMBER	0002	
ACTION_OPENED  . . . . . . . . .  	NUMBER	0001	
ACTION_REPLACED_OPENED . . . . .  	NUMBER	0003	
ADDR_INT_ABORT . . . . . . . . .  	NUMBER	0080	
ADDR_INT_COMMAND . . . . . . . .  	NUMBER	0084	
ADDR_INT_CTRL_C  . . . . . . . .  	NUMBER	008C	
ADDR_INT_DISK_READ . . . . . . .  	NUMBER	0094	
ADDR_INT_DISK_WRITE  . . . . . .  	NUMBER	0098	
ADDR_INT_FASTCON . . . . . . . .  	NUMBER	00A4	
ADDR_INT_FATAL_ABORT . . . . . .  	NUMBER	0090	
ADDR_INT_IBM . . . . . . . . . .  	NUMBER	00A8	
ADDR_INT_KEEP_PROCESS  . . . . .  	NUMBER	009C	
ADDR_INT_SPOOLER . . . . . . . .  	NUMBER	00A0	
ADDR_INT_TERMINATE . . . . . . .  	NUMBER	0088	
ALLOC  . . . . . . . . . . . . .  	NUMBER	0048	
ALLOCOPER  . . . . . . . . . . .  	NUMBER	0058	
ALLOWED_FAIL . . . . . . . . . .  	NUMBER	0008	
ALLOWED_IGNORE . . . . . . . . .  	NUMBER	0020	
ALLOWED_RETRY  . . . . . . . . .  	NUMBER	0010	
ALTVECT  . . . . . . . . . . . .  	ALIAS	 FALSE		
ALT_EXPECTED_VERSION . . . . . .  	NUMBER	1A05	
ALT_MAJOR_VERSION  . . . . . . .  	NUMBER	0005	
ALT_MINOR_VERSION  . . . . . . .  	NUMBER	001A	
ARENA_OWNER_SYSTEM . . . . . . .  	NUMBER	0000	
ARENA_SIGNATURE_END  . . . . . .  	NUMBER	005A	
ARENA_SIGNATURE_NORMAL . . . . .  	NUMBER	004D	
ARG_BUF_INDEX  . . . . . . . . .  	L WORD	047C	DATA	Global
ASMADD . . . . . . . . . . . . .  	L BYTE	0459	DATA	Global	Length = 0004
ASMSP  . . . . . . . . . . . . .  	L WORD	0463	DATA	Global
ASSEM1 . . . . . . . . . . . . .  	L BYTE	048B	DATA	Global
ASSEM2 . . . . . . . . . . . . .  	L BYTE	048C	DATA	Global
ASSEM3 . . . . . . . . . . . . .  	L BYTE	048D	DATA	Global
ASSEM4 . . . . . . . . . . . . .  	L BYTE	048E	DATA	Global
ASSEM5 . . . . . . . . . . . . .  	L BYTE	048F	DATA	Global
ASSEM6 . . . . . . . . . . . . .  	L BYTE	0490	DATA	Global
ASSEM_CNT  . . . . . . . . . . .  	L BYTE	048A	DATA	Global
ASSIGNOPER . . . . . . . . . . .  	NUMBER	005F	
ATTR_ALL . . . . . . . . . . . .  	NUMBER	0016	
ATTR_ARCHIVE . . . . . . . . . .  	NUMBER	0020	
ATTR_CHANGEABLE  . . . . . . . .  	NUMBER	0027	
ATTR_DEVICE  . . . . . . . . . .  	NUMBER	0040	
ATTR_DIRECTORY . . . . . . . . .  	NUMBER	0010	
ATTR_HIDDEN  . . . . . . . . . .  	NUMBER	0002	
ATTR_IGNORE  . . . . . . . . . .  	NUMBER	0061	
ATTR_READ_ONLY . . . . . . . . .  	NUMBER	0001	
ATTR_SYSTEM  . . . . . . . . . .  	NUMBER	0004	
ATTR_VOLUME_ID . . . . . . . . .  	NUMBER	0008	
AUTO_COMMIT_WRITE  . . . . . . .  	NUMBER	4000	
AWORD  . . . . . . . . . . . . .  	L BYTE	0480	DATA	Global

BEGSEG . . . . . . . . . . . . .  	L WORD	0475	DATA	Global
BPFLG  . . . . . . . . . . . . .  	L BYTE	0516	DATA	Global
BPINTSAV . . . . . . . . . . . .  	L DWORD	0432	DATA	Global
BPLEN  . . . . . . . . . . . . .  	NUMBER	0032	
BPMAX  . . . . . . . . . . . . .  	NUMBER	000A	
BPREG  . . . . . . . . . . . . .  	NUMBER	5042	
BPTAB  . . . . . . . . . . . . .  	L BYTE	04E1	DATA	Global	Length = 0032
BRKCNT . . . . . . . . . . . . .  	L WORD	0486	DATA	Global
BUFFER . . . . . . . . . . . . .  	L BYTE	047B	DATA	Global
BUFFERFLAG . . . . . . . . . . .  	NUMBER	FFFF	
BUFINSIZ . . . . . . . . . . . .  	NUMBER	0014	
BUFLEN . . . . . . . . . . . . .  	NUMBER	0050	
BUFSIZ . . . . . . . . . . . . .  	NUMBER	0200	
BUF_DIRTY  . . . . . . . . . . .  	NUMBER	0040	
BUF_DPB  . . . . . . . . . . . .  		000D	
BUF_FILL . . . . . . . . . . . .  		0011	
BUF_FLAGS  . . . . . . . . . . .  		0005	
BUF_FREE . . . . . . . . . . . .  	NUMBER	00FF	
BUF_ID . . . . . . . . . . . . .  		0004	
BUF_ISDATA . . . . . . . . . . .  	NUMBER	0008	
Microsoft (R) Macro Assembler Version 5.10                  2/14/25 23:44:19
DEBDATA.SAL - PC DOS                                        Symbols-6


BUF_ISDIR  . . . . . . . . . . .  	NUMBER	0004	
BUF_ISFAT  . . . . . . . . . . .  	NUMBER	0002	
BUF_ISNET  . . . . . . . . . . .  	NUMBER	0080	
BUF_NETID  . . . . . . . . . . .  	ALIAS	 BUFINSIZ		
BUF_NEXT . . . . . . . . . . . .  		0000	
BUF_OFFSET . . . . . . . . . . .  	DWORD	0006	
BUF_PREV . . . . . . . . . . . .  		0002	
BUF_RESERVED . . . . . . . . . .  		0013	
BUF_SECTOR . . . . . . . . . . .  		0006	
BUF_SNBUF  . . . . . . . . . . .  	NUMBER	0010	
BUF_TYPE_0 . . . . . . . . . . .  	NUMBER	00F1	
BUF_VISIT  . . . . . . . . . . .  	NUMBER	0020	
BUF_WRTCNT . . . . . . . . . . .  		000A	
BUF_WRTCNTINC  . . . . . . . . .  		000B	
BXFLG  . . . . . . . . . . . . .  	L BYTE	0515	DATA	Global
BXREG  . . . . . . . . . . . . .  	NUMBER	5842	
BYTCNT . . . . . . . . . . . . .  	L BYTE	047B	DATA	Global
BYTEBUF  . . . . . . . . . . . .  	L BYTE	0491	DATA	Global	Length = 0050

CARGS  . . . . . . . . . . . . .  	NUMBER	0000	
CHAR_AT_SIGN . . . . . . . . . .  	NUMBER	0040	
CHAR_BACKSPACE . . . . . . . . .  	NUMBER	0008	
CHAR_BLANK . . . . . . . . . . .  	NUMBER	0020	
CHAR_COLON . . . . . . . . . . .  	NUMBER	003A	
CHAR_COMMA . . . . . . . . . . .  	NUMBER	002C	
CHAR_EOF . . . . . . . . . . . .  	NUMBER	001A	
CHAR_EQUAL . . . . . . . . . . .  	NUMBER	003D	
CHAR_LEFT_BRACKET  . . . . . . .  	NUMBER	005B	
CHAR_MINUS . . . . . . . . . . .  	NUMBER	002D	
CHAR_OPER  . . . . . . . . . . .  	NUMBER	0037	
CHAR_PERIOD  . . . . . . . . . .  	NUMBER	002E	
CHAR_RUBOUT  . . . . . . . . . .  	NUMBER	007F	
CHAR_SEMICOLON . . . . . . . . .  	NUMBER	003B	
CHAR_TAB . . . . . . . . . . . .  	NUMBER	0009	
CHAR_ZERO  . . . . . . . . . . .  	NUMBER	0030	
CHDIR  . . . . . . . . . . . . .  	NUMBER	003B	
CHMOD  . . . . . . . . . . . . .  	NUMBER	0043	
CLOSE  . . . . . . . . . . . . .  	NUMBER	003E	
COMMA  . . . . . . . . . . . . .  	NUMBER	2C00	
COMMIT . . . . . . . . . . . . .  	NUMBER	0068	
CR . . . . . . . . . . . . . . .  	NUMBER	000D	
CREAT  . . . . . . . . . . . . .  	NUMBER	003C	
CREATENEWFILE  . . . . . . . . .  	NUMBER	005B	
CREATETEMPFILE . . . . . . . . .  	NUMBER	005A	
CREATE_LONG  . . . . . . . . . .  	L DWORD	0473	DATA	Global
CREATE_PROCESS_DATA_BLOCK  . . .  	NUMBER	0026	
CRITASSIGN . . . . . . . . . . .  	NUMBER	0008	
CRITDEVICE . . . . . . . . . . .  	NUMBER	0002	
CRITDISK . . . . . . . . . . . .  	NUMBER	0001	
CRITIFS  . . . . . . . . . . . .  	NUMBER	0006	
CRITMEM  . . . . . . . . . . . .  	NUMBER	0001	
CRITNET  . . . . . . . . . . . .  	NUMBER	0005	
CRITSFT  . . . . . . . . . . . .  	NUMBER	0001	
CRITSHARE  . . . . . . . . . . .  	NUMBER	0001	
CURDIRLEN  . . . . . . . . . . .  	NUMBER	0058	
CURDIR_INUSE . . . . . . . . . .  	NUMBER	4000	
CURDIR_ISIFS . . . . . . . . . .  	NUMBER	8000	
CURDIR_ISNET . . . . . . . . . .  	NUMBER	8000	
CURDIR_LOCAL . . . . . . . . . .  	NUMBER	1000	
CURDIR_NETID . . . . . . . . . .  	DWORD	0049	
CURDIR_SPLICE  . . . . . . . . .  	NUMBER	2000	
CURRENT_DIR  . . . . . . . . . .  	NUMBER	0047	
C_BS . . . . . . . . . . . . . .  	NUMBER	0008	
C_CR . . . . . . . . . . . . . .  	NUMBER	000D	
C_DEL  . . . . . . . . . . . . .  	NUMBER	007F	
C_ETB  . . . . . . . . . . . . .  	NUMBER	0017	
C_ETX  . . . . . . . . . . . . .  	NUMBER	0003	
C_HT . . . . . . . . . . . . . .  	NUMBER	0009	
C_LF . . . . . . . . . . . . . .  	NUMBER	000A	
C_NAK  . . . . . . . . . . . . .  	NUMBER	0015	

DATAEND  . . . . . . . . . . . .  	L WORD	067B	DATA	Global
DBCS . . . . . . . . . . . . . .  	NUMBER	0000	
DEALLOC  . . . . . . . . . . . .  	NUMBER	0049	
DEBUG  . . . . . . . . . . . . .  	NUMBER	0000	
DEFDUMP  . . . . . . . . . . . .  	L BYTE	0467	DATA	Global	Length = 0004
Microsoft (R) Macro Assembler Version 5.10                  2/14/25 23:44:19
DEBDATA.SAL - PC DOS                                        Symbols-7


DEFLEN . . . . . . . . . . . . .  	L WORD	046B	DATA	Global
DEVID_BLOCK_DEV  . . . . . . . .  	NUMBER	001F	
DEVID_DEVICE . . . . . . . . . .  	NUMBER	0080	
DEVID_DEVICE_CLOCK . . . . . . .  	NUMBER	0008	
DEVID_DEVICE_CON_IN  . . . . . .  	NUMBER	0001	
DEVID_DEVICE_CON_OUT . . . . . .  	NUMBER	0002	
DEVID_DEVICE_EOF . . . . . . . .  	NUMBER	0040	
DEVID_DEVICE_NULL  . . . . . . .  	NUMBER	0004	
DEVID_DEVICE_RAW . . . . . . . .  	NUMBER	0020	
DEVID_DEVICE_SPECIAL . . . . . .  	NUMBER	0010	
DEVID_EOF  . . . . . . . . . . .  	NUMBER	0040	
DEVID_FILE_CLEAN . . . . . . . .  	NUMBER	0040	
DEVID_FILE_MASK_DRIVE  . . . . .  	NUMBER	003F	
DEVID_ISCIN  . . . . . . . . . .  	NUMBER	0001	
DEVID_ISCLK  . . . . . . . . . .  	NUMBER	0008	
DEVID_ISCOT  . . . . . . . . . .  	NUMBER	0002	
DEVID_ISDEV  . . . . . . . . . .  	NUMBER	0080	
DEVID_ISNUL  . . . . . . . . . .  	NUMBER	0004	
DEVID_RAW  . . . . . . . . . . .  	NUMBER	0020	
DEVID_SPECIAL  . . . . . . . . .  	NUMBER	0010	
DIFLG  . . . . . . . . . . . . .  	L BYTE	0513	DATA	Global
DIREG  . . . . . . . . . . . . .  	NUMBER	4944	
DIRFLG . . . . . . . . . . . . .  	L BYTE	0523	DATA	Global
DIRSTRLEN  . . . . . . . . . . .  	NUMBER	0043	
DIR_SEARCH_FIRST . . . . . . . .  	NUMBER	0011	
DIR_SEARCH_NEXT  . . . . . . . .  	NUMBER	0012	
DISADD . . . . . . . . . . . . .  	L BYTE	045D	DATA	Global	Length = 0004
DISCNT . . . . . . . . . . . . .  	L WORD	0461	DATA	Global
DISK_RESET . . . . . . . . . . .  	NUMBER	000D	
DOUBLE_QUOTE . . . . . . . . . .  	NUMBER	0022	
DPBSIZ . . . . . . . . . . . . .  	NUMBER	0021	
DSKSIZ . . . . . . . . . . . . .  	NUMBER	000D	
DUP_PDB  . . . . . . . . . . . .  	NUMBER	0055	

ECS_CALL . . . . . . . . . . . .  	NUMBER	0063	
EMS_GET_MAN_STAT . . . . . . . .  	NUMBER	0040	
EMS_GET_PAGE_MAP . . . . . . . .  	NUMBER	0000	
EMS_GET_SET_PG_MP  . . . . . . .  	NUMBER	004E	
EMS_HANDLE_CNT . . . . . . . . .  	NUMBER	004B	
EMS_HANDLE_PAGES . . . . . . . .  	NUMBER	004D	
EMS_HANDLE_TOTAL . . . . . . . .  	NUMBER	00FF	
EMS_HAN_ALLOC  . . . . . . . . .  	NUMBER	0043	
EMS_LIM_40 . . . . . . . . . . .  	NUMBER	0040	
EMS_MAP_BUFF_SIZE  . . . . . . .  	NUMBER	000C	
EMS_MAP_MEMORY . . . . . . . . .  	NUMBER	0044	
EMS_PAGE_DEALL . . . . . . . . .  	NUMBER	0045	
EMS_PG_FRAME . . . . . . . . . .  	NUMBER	5800	
EMS_REST_PAGE_MAP  . . . . . . .  	NUMBER	0048	
EMS_SAVE_PAGE_MAP  . . . . . . .  	NUMBER	0047	
EMS_SET_PAGE_MAP . . . . . . . .  	NUMBER	0001	
EMS_UNALL_PG_CNT . . . . . . . .  	NUMBER	0042	
EMS_VERSION  . . . . . . . . . .  	NUMBER	0046	
ENTRYPOINT . . . . . . . . . . .  	NUMBER	00C0	
ERRACT_ABORT . . . . . . . . . .  	NUMBER	0004	
ERRACT_DLYRET  . . . . . . . . .  	NUMBER	0002	
ERRACT_IGNORE  . . . . . . . . .  	NUMBER	0006	
ERRACT_INTRET  . . . . . . . . .  	NUMBER	0007	
ERRACT_PANIC . . . . . . . . . .  	NUMBER	0005	
ERRACT_RETRY . . . . . . . . . .  	NUMBER	0001	
ERRACT_USER  . . . . . . . . . .  	NUMBER	0003	
ERRCLASS_ALREADY . . . . . . . .  	NUMBER	000C	
ERRCLASS_APPERR  . . . . . . . .  	NUMBER	0007	
ERRCLASS_AUTH  . . . . . . . . .  	NUMBER	0003	
ERRCLASS_BADFMT  . . . . . . . .  	NUMBER	0009	
ERRCLASS_HRDFAIL . . . . . . . .  	NUMBER	0005	
ERRCLASS_INTRN . . . . . . . . .  	NUMBER	0004	
ERRCLASS_LOCKED  . . . . . . . .  	NUMBER	000A	
ERRCLASS_MEDIA . . . . . . . . .  	NUMBER	000B	
ERRCLASS_NOTFND  . . . . . . . .  	NUMBER	0008	
ERRCLASS_OUTRES  . . . . . . . .  	NUMBER	0001	
ERRCLASS_SYSFAIL . . . . . . . .  	NUMBER	0006	
ERRCLASS_TEMPSIT . . . . . . . .  	NUMBER	0002	
ERRCLASS_UNK . . . . . . . . . .  	NUMBER	000D	
ERRLOC_DISK  . . . . . . . . . .  	NUMBER	0002	
ERRLOC_MEM . . . . . . . . . . .  	NUMBER	0005	
ERRLOC_NET . . . . . . . . . . .  	NUMBER	0003	
Microsoft (R) Macro Assembler Version 5.10                  2/14/25 23:44:19
DEBDATA.SAL - PC DOS                                        Symbols-8


ERRLOC_SERDEV  . . . . . . . . .  	NUMBER	0004	
ERRLOC_UNK . . . . . . . . . . .  	NUMBER	0001	
ERROR_ACCESS_DENIED  . . . . . .  	NUMBER	0005	
ERROR_ALREADY_ASSIGNED . . . . .  	NUMBER	0055	
ERROR_ARENA_TRASHED  . . . . . .  	NUMBER	0007	
ERROR_BAD_COMMAND  . . . . . . .  	NUMBER	0016	
ERROR_BAD_ENVIRONMENT  . . . . .  	NUMBER	000A	
ERROR_BAD_FORMAT . . . . . . . .  	NUMBER	000B	
ERROR_BAD_LENGTH . . . . . . . .  	NUMBER	0018	
ERROR_BAD_UNIT . . . . . . . . .  	NUMBER	0014	
ERROR_CANNOT_MAKE  . . . . . . .  	NUMBER	0052	
ERROR_CODE_PAGE_MISMATCHED . . .  	NUMBER	0025	
ERROR_CRC  . . . . . . . . . . .  	NUMBER	0017	
ERROR_CURRENT_DIRECTORY  . . . .  	NUMBER	0010	
ERROR_DUP_FCB  . . . . . . . . .  	NUMBER	0051	
ERROR_FAIL_I24 . . . . . . . . .  	NUMBER	0053	
ERROR_FCB_UNAVAILABLE  . . . . .  	NUMBER	0023	
ERROR_FILE_EXISTS  . . . . . . .  	NUMBER	0050	
ERROR_FILE_NOT_FOUND . . . . . .  	NUMBER	0002	
ERROR_GEN_FAILURE  . . . . . . .  	NUMBER	001F	
ERROR_HANDLE_DISK_FULL . . . . .  	NUMBER	0027	
ERROR_HANDLE_EOF . . . . . . . .  	NUMBER	0026	
ERROR_I24_BAD_COMMAND  . . . . .  	NUMBER	0003	
ERROR_I24_BAD_LENGTH . . . . . .  	NUMBER	0005	
ERROR_I24_BAD_UNIT . . . . . . .  	NUMBER	0001	
ERROR_I24_CRC  . . . . . . . . .  	NUMBER	0004	
ERROR_I24_GEN_FAILURE  . . . . .  	NUMBER	000C	
ERROR_I24_NOT_DOS_DISK . . . . .  	NUMBER	0007	
ERROR_I24_NOT_READY  . . . . . .  	NUMBER	0002	
ERROR_I24_OUT_OF_PAPER . . . . .  	NUMBER	0009	
ERROR_I24_READ_FAULT . . . . . .  	NUMBER	000B	
ERROR_I24_SECTOR_NOT_FOUND . . .  	NUMBER	0008	
ERROR_I24_SEEK . . . . . . . . .  	NUMBER	0006	
ERROR_I24_WRITE_FAULT  . . . . .  	NUMBER	000A	
ERROR_I24_WRITE_PROTECT  . . . .  	NUMBER	0000	
ERROR_I24_WRONG_DISK . . . . . .  	NUMBER	000F	
ERROR_INVALID_ACCESS . . . . . .  	NUMBER	000C	
ERROR_INVALID_BLOCK  . . . . . .  	NUMBER	0009	
ERROR_INVALID_DATA . . . . . . .  	NUMBER	000D	
ERROR_INVALID_DRIVE  . . . . . .  	NUMBER	000F	
ERROR_INVALID_FUNCTION . . . . .  	NUMBER	0001	
ERROR_INVALID_HANDLE . . . . . .  	NUMBER	0006	
ERROR_INVALID_PARAMETER  . . . .  	NUMBER	0057	
ERROR_INVALID_PASSWORD . . . . .  	NUMBER	0056	
ERROR_LOCK_VIOLATION . . . . . .  	NUMBER	0021	
ERROR_NET_WRITE_FAULT  . . . . .  	NUMBER	0058	
ERROR_NOT_DOS_DISK . . . . . . .  	NUMBER	001A	
ERROR_NOT_ENOUGH_MEMORY  . . . .  	NUMBER	0008	
ERROR_NOT_READY  . . . . . . . .  	NUMBER	0015	
ERROR_NOT_SAME_DEVICE  . . . . .  	NUMBER	0011	
ERROR_NOT_SUPPORTED  . . . . . .  	NUMBER	0032	
ERROR_NO_MORE_FILES  . . . . . .  	NUMBER	0012	
ERROR_OUT_OF_PAPER . . . . . . .  	NUMBER	001C	
ERROR_OUT_OF_STRUCTURES  . . . .  	NUMBER	0054	
ERROR_PATH_NOT_FOUND . . . . . .  	NUMBER	0003	
ERROR_READ_FAULT . . . . . . . .  	NUMBER	001E	
ERROR_SECTOR_NOT_FOUND . . . . .  	NUMBER	001B	
ERROR_SEEK . . . . . . . . . . .  	NUMBER	0019	
ERROR_SHARING_BUFFER_EXCEEDED  .  	NUMBER	0024	
ERROR_SHARING_VIOLATION  . . . .  	NUMBER	0020	
ERROR_SYS_COMP_NOT_LOADED  . . .  	NUMBER	005A	
ERROR_TOO_MANY_OPEN_FILES  . . .  	NUMBER	0004	
ERROR_WRITE_FAULT  . . . . . . .  	NUMBER	001D	
ERROR_WRITE_PROTECT  . . . . . .  	NUMBER	0013	
ERROR_WRONG_DISK . . . . . . . .  	NUMBER	0022	
EXEC . . . . . . . . . . . . . .  	NUMBER	004B	
EXEC_FUNC_NO_EXECUTE . . . . . .  	NUMBER	0001	
EXEC_FUNC_OVERLAY  . . . . . . .  	NUMBER	0002	
EXEFCB . . . . . . . . . . . . .  	ALIAS	 FCB		
EXE_VALID_OLD_SIGNATURE  . . . .  	NUMBER	4D5A	
EXE_VALID_SIGNATURE  . . . . . .  	NUMBER	5A4D	
EXISTS_MASK  . . . . . . . . . .  	NUMBER	000F	
EXIT . . . . . . . . . . . . . .  	NUMBER	004C	
EXIT_ABORT . . . . . . . . . . .  	NUMBER	0000	
EXIT_CTRL_C  . . . . . . . . . .  	NUMBER	0001	
EXIT_HARD_ERROR  . . . . . . . .  	NUMBER	0002	
Microsoft (R) Macro Assembler Version 5.10                  2/14/25 23:44:19
DEBDATA.SAL - PC DOS                                        Symbols-9


EXIT_KEEP_PROCESS  . . . . . . .  	NUMBER	0003	
EXIT_TERMINATE . . . . . . . . .  	NUMBER	0000	
EXPECTED_VERSION . . . . . . . .  	NUMBER	0004	
EXTHANDLE  . . . . . . . . . . .  	NUMBER	0067	
EXTOPEN  . . . . . . . . . . . .  	NUMBER	006C	
EXTPTR . . . . . . . . . . . . .  	L WORD	0450	DATA	Global
EXT_EXISTS_FAIL  . . . . . . . .  	NUMBER	0000	
EXT_EXISTS_OPEN  . . . . . . . .  	NUMBER	0001	
EXT_FILE_NOT_EXISTS  . . . . . .  	NUMBER	0004	
EXT_NEXISTS_CREATE . . . . . . .  	NUMBER	0010	
EXT_OPEN_I24_OFF . . . . . . . .  	NUMBER	0002	
EXT_OPEN_ON  . . . . . . . . . .  	NUMBER	0001	

F8087  . . . . . . . . . . . . .  	L BYTE	0522	DATA	Global
FALSE  . . . . . . . . . . . . .  	NUMBER	0000	
FCB  . . . . . . . . . . . . . .  	NUMBER	005C	
FCBDEVICE  . . . . . . . . . . .  	NUMBER	0040	
FCBMASK  . . . . . . . . . . . .  	NUMBER	00C0	
FCBNETWORK . . . . . . . . . . .  	NUMBER	0080	
FCBSHARE . . . . . . . . . . . .  	NUMBER	00C0	
FCBSPECIAL . . . . . . . . . . .  	NUMBER	0080	
FCB_CLOSE  . . . . . . . . . . .  	NUMBER	0010	
FCB_CREATE . . . . . . . . . . .  	NUMBER	0016	
FCB_DELETE . . . . . . . . . . .  	NUMBER	0013	
FCB_L_ATTR . . . . . . . . . . .  	BYTE	001E	
FCB_L_DRIVE  . . . . . . . . . .  	BYTE	0019	
FCB_L_FIRCLUS  . . . . . . . . .  	WORD	001A	
FCB_L_MFS  . . . . . . . . . . .  	WORD	001C	
FCB_NETID  . . . . . . . . . . .  	DWORD	001C	
FCB_NET_DRIVE  . . . . . . . . .  	BYTE	0019	
FCB_NET_HANDLE . . . . . . . . .  	WORD	001A	
FCB_NSLD_DRIVE . . . . . . . . .  	BYTE	0019	
FCB_NSLD_DRVPTR  . . . . . . . .  	DWORD	001A	
FCB_NSL_BITS . . . . . . . . . .  	BYTE	001A	
FCB_NSL_DIRPOS . . . . . . . . .  	BYTE	001F	
FCB_NSL_DIRSEC . . . . . . . . .  	WORD	001D	
FCB_NSL_DRIVE  . . . . . . . . .  	BYTE	0019	
FCB_NSL_FIRCLUS  . . . . . . . .  	WORD	001B	
FCB_OPEN . . . . . . . . . . . .  	NUMBER	000F	
FCB_RANDOM_READ  . . . . . . . .  	NUMBER	0021	
FCB_RANDOM_READ_BLOCK  . . . . .  	NUMBER	0027	
FCB_RANDOM_WRITE . . . . . . . .  	NUMBER	0022	
FCB_RANDOM_WRITE_BLOCK . . . . .  	NUMBER	0028	
FCB_RENAME . . . . . . . . . . .  	NUMBER	0017	
FCB_SEQ_READ . . . . . . . . . .  	NUMBER	0014	
FCB_SEQ_WRITE  . . . . . . . . .  	NUMBER	0015	
FCB_SFN  . . . . . . . . . . . .  	BYTE	0018	
FCHK . . . . . . . . . . . . . .  	NUMBER	0001	
FDELIM . . . . . . . . . . . . .  	NUMBER	0002	
FFCB . . . . . . . . . . . . . .  	NUMBER	0008	
FILDIRENT  . . . . . . . . . . .  	NUMBER	0010	
FILEEND  . . . . . . . . . . . .  	L WORD	042A	DATA	Global
FILESTRT . . . . . . . . . . . .  	L WORD	042C	DATA	Global
FILE_TIMES . . . . . . . . . . .  	NUMBER	0057	
FILPERPROC . . . . . . . . . . .  	NUMBER	0014	
FIN24  . . . . . . . . . . . . .  	L BYTE	0428	DATA	Global
FIND_FIRST . . . . . . . . . . .  	NUMBER	004E	
FIND_NEXT  . . . . . . . . . . .  	NUMBER	004F	
FSPCHK . . . . . . . . . . . . .  	NUMBER	0004	
FZTRACE  . . . . . . . . . . . .  	L BYTE	0429	DATA	Global
F_AUX  . . . . . . . . . . . . .  	NUMBER	0010	
F_CARRY  . . . . . . . . . . . .  	NUMBER	0001	
F_DIRECTION  . . . . . . . . . .  	NUMBER	0400	
F_INTERRUPT  . . . . . . . . . .  	NUMBER	0200	
F_OVERFLOW . . . . . . . . . . .  	NUMBER	0800	
F_PARITY . . . . . . . . . . . .  	NUMBER	0004	
F_SIGN . . . . . . . . . . . . .  	NUMBER	0080	
F_TRACE  . . . . . . . . . . . .  	NUMBER	0100	
F_ZERO . . . . . . . . . . . . .  	NUMBER	0040	

GENERIC_IOCTL  . . . . . . . . .  	NUMBER	440D	
GETCURRENTPSP  . . . . . . . . .  	NUMBER	0062	
GETEXTCNTRY  . . . . . . . . . .  	NUMBER	0065	
GETEXTENDEDERROR . . . . . . . .  	NUMBER	0059	
GETSETCDPG . . . . . . . . . . .  	NUMBER	0066	
GETSETMEDIAID  . . . . . . . . .  	NUMBER	0069	
Microsoft (R) Macro Assembler Version 5.10                  2/14/25 23:44:19
DEBDATA.SAL - PC DOS                                        Symbols-10


GET_CURRENT_PDB  . . . . . . . .  	NUMBER	0051	
GET_DATE . . . . . . . . . . . .  	NUMBER	002A	
GET_DEFAULT_DPB  . . . . . . . .  	NUMBER	001F	
GET_DEFAULT_DRIVE  . . . . . . .  	NUMBER	0019	
GET_DMA  . . . . . . . . . . . .  	NUMBER	002F	
GET_DPB  . . . . . . . . . . . .  	NUMBER	0032	
GET_DRIVE_FREESPACE  . . . . . .  	NUMBER	0036	
GET_FCB_FILE_LENGTH  . . . . . .  	NUMBER	0023	
GET_FCB_POSITION . . . . . . . .  	NUMBER	0024	
GET_INDOS_FLAG . . . . . . . . .  	NUMBER	0034	
GET_INTERRUPT_VECTOR . . . . . .  	NUMBER	0035	
GET_IN_VARS  . . . . . . . . . .  	NUMBER	0052	
GET_TIME . . . . . . . . . . . .  	NUMBER	002C	
GET_VERIFY_ON_WRITE  . . . . . .  	NUMBER	0054	
GET_VERSION  . . . . . . . . . .  	NUMBER	0030	

HANDLE . . . . . . . . . . . . .  	L WORD	0452	DATA	Global
HANDLE_FAIL_I24  . . . . . . . .  	NUMBER	0100	
HINUM  . . . . . . . . . . . . .  	L WORD	0520	DATA	Global
HONGEUL  . . . . . . . . . . . .  	NUMBER	0063	

I24_AREA . . . . . . . . . . . .  	NUMBER	0006	
I24_CLASS  . . . . . . . . . . .  	NUMBER	0080	
I24_OPERATION  . . . . . . . . .  	NUMBER	0001	
IBM  . . . . . . . . . . . . . .  	ALIAS	 IBMVER		
IBMCOPYRIGHT . . . . . . . . . .  	ALIAS	 FALSE		
IBMJAPAN . . . . . . . . . . . .  	ALIAS	 FALSE		
IBMJAPVER  . . . . . . . . . . .  	ALIAS	 FALSE		
IBMVER . . . . . . . . . . . . .  	ALIAS	 TRUE		
IFS_IOCTL  . . . . . . . . . . .  	NUMBER	006B	
INDEX  . . . . . . . . . . . . .  	L WORD	0465	DATA	Global
INSTALLED  . . . . . . . . . . .  	NUMBER	FFFF	
INSTALLEDDATA  . . . . . . . . .  	NUMBER	0000	
INTBASE  . . . . . . . . . . . .  	NUMBER	0080	
INTERNAT . . . . . . . . . . . .  	ALIAS	 FALSE		
INTERNATIONAL  . . . . . . . . .  	NUMBER	0038	
INTERNAT_BLOCK_MAX . . . . . . .  	NUMBER	0020	
INTTAB . . . . . . . . . . . . .  	NUMBER	0020	
INT_24_ERROR . . . . . . . . . .  	NUMBER	2000	
INT_ABORT  . . . . . . . . . . .  	ALIAS	 INTTAB		
INT_COMMAND  . . . . . . . . . .  	NUMBER	0021	
INT_CTRL_C . . . . . . . . . . .  	NUMBER	0023	
INT_DISK_READ  . . . . . . . . .  	NUMBER	0025	
INT_DISK_WRITE . . . . . . . . .  	NUMBER	0026	
INT_FASTCON  . . . . . . . . . .  	NUMBER	0029	
INT_FATAL_ABORT  . . . . . . . .  	NUMBER	0024	
INT_IBM  . . . . . . . . . . . .  	NUMBER	002A	
INT_KEEP_PROCESS . . . . . . . .  	NUMBER	0027	
INT_MASK . . . . . . . . . . . .  	NUMBER	00FF	
INT_SPOOLER  . . . . . . . . . .  	NUMBER	0028	
INT_TERMINATE  . . . . . . . . .  	NUMBER	0022	
IOCTL  . . . . . . . . . . . . .  	NUMBER	0044	
IO_MODE_ID . . . . . . . . . . .  	NUMBER	0002	

JAPAN  . . . . . . . . . . . . .  	ALIAS	 FALSE		

KANJI  . . . . . . . . . . . . .  	ALIAS	 FALSE		
KEEP_PROCESS . . . . . . . . . .  	NUMBER	0031	
KOREA  . . . . . . . . . . . . .  	ALIAS	 FALSE		

lbtbl  . . . . . . . . . . . . .  	L DWORD	000A	DATA	Global
LF . . . . . . . . . . . . . . .  	NUMBER	000A	
LOCKOPER . . . . . . . . . . . .  	NUMBER	005C	
LOWER_A  . . . . . . . . . . . .  	NUMBER	0061	
LOWER_Z  . . . . . . . . . . . .  	NUMBER	007A	
LOWNUM . . . . . . . . . . . . .  	L WORD	051E	DATA	Global
LSEEK  . . . . . . . . . . . . .  	NUMBER	0042	
LSEEK_EOF_OPTION . . . . . . . .  	NUMBER	0002	
LSEEK_FROM_START . . . . . . . .  	NUMBER	0000	

MAJOR_VERSION  . . . . . . . . .  	NUMBER	0004	
MASK_PORT  . . . . . . . . . . .  	NUMBER	0021	
MAXBUCKETINPAGE  . . . . . . . .  	NUMBER	0002	
MAXBUFFINBUCKET  . . . . . . . .  	NUMBER	000F	
MEMFLG . . . . . . . . . . . . .  	L BYTE	0519	DATA	Global
MEMS . . . . . . . . . . . . . .  	NUMBER	0001	
Microsoft (R) Macro Assembler Version 5.10                  2/14/25 23:44:19
DEBDATA.SAL - PC DOS                                        Symbols-11


MIDFLD . . . . . . . . . . . . .  	L BYTE	0482	DATA	Global
MINOR_VERSION  . . . . . . . . .  	NUMBER	0000	
MI_INT . . . . . . . . . . . . .  	NUMBER	00CD	
MI_LONG_CALL . . . . . . . . . .  	NUMBER	009A	
MI_LONG_JMP  . . . . . . . . . .  	NUMBER	00EA	
MI_LONG_RET  . . . . . . . . . .  	NUMBER	00CB	
MI_NEAR_RET  . . . . . . . . . .  	NUMBER	00C3	
MKDIR  . . . . . . . . . . . . .  	NUMBER	0039	
MODE . . . . . . . . . . . . . .  	L BYTE	0483	DATA	Global
MOVFLG . . . . . . . . . . . . .  	L BYTE	051B	DATA	Global
MSVER  . . . . . . . . . . . . .  	NUMBER	0000	
MULTDOS  . . . . . . . . . . . .  	NUMBER	0012	
MULTIFS  . . . . . . . . . . . .  	NUMBER	0011	
MULTNET  . . . . . . . . . . . .  	NUMBER	0011	
MULTSHARE  . . . . . . . . . . .  	NUMBER	0010	

NEGFLG . . . . . . . . . . . . .  	L BYTE	0517	DATA	Global
NLSFUNC  . . . . . . . . . . . .  	NUMBER	0014	
NOT_EXISTS_MASK  . . . . . . . .  	NUMBER	00F0	
NO_CODE_PAGE_CHECK . . . . . . .  	NUMBER	0100	
NSEG . . . . . . . . . . . . . .  	L WORD	0484	DATA	Global
NUMFLG . . . . . . . . . . . . .  	L BYTE	0518	DATA	Global

OEM_C1 . . . . . . . . . . . . .  	NUMBER	00F9	
OEM_C2 . . . . . . . . . . . . .  	NUMBER	00FA	
OEM_C3 . . . . . . . . . . . . .  	NUMBER	00FB	
OEM_C4 . . . . . . . . . . . . .  	NUMBER	00FC	
OEM_C5 . . . . . . . . . . . . .  	NUMBER	00FD	
OEM_C6 . . . . . . . . . . . . .  	NUMBER	00FE	
OEM_C7 . . . . . . . . . . . . .  	NUMBER	00FF	
OFFSAVE  . . . . . . . . . . . .  	L WORD	0471	DATA	Global
OLD_MASK . . . . . . . . . . . .  	L BYTE	0423	DATA	Global
OPBUFLEN . . . . . . . . . . . .  	NUMBER	0023	
OPCODE . . . . . . . . . . . . .  	L WORD	047E	DATA	Global
OPEN . . . . . . . . . . . . . .  	NUMBER	003D	
OPEN_FOR_BOTH  . . . . . . . . .  	NUMBER	0002	
OPEN_FOR_READ  . . . . . . . . .  	NUMBER	0000	
OPEN_FOR_WRITE . . . . . . . . .  	NUMBER	0001	

PARITYFLAG . . . . . . . . . . .  	L BYTE	0436	DATA	Global
PARSERR  . . . . . . . . . . . .  	L BYTE	0458	DATA	Global
PARSE_FILE_DESCRIPTOR  . . . . .  	NUMBER	0029	
PATHPARSE  . . . . . . . . . . .  	NUMBER	0061	
PDB_APPEND . . . . . . . . . . .  	BYTE	003D	
PDB_INTERCON . . . . . . . . . .  	BYTE	003C	
PREV24 . . . . . . . . . . . . .  	L DWORD	0424	DATA	Global
PROMPT . . . . . . . . . . . . .  	NUMBER	002D	

RAW_CON_INPUT  . . . . . . . . .  	NUMBER	0007	
RAW_CON_IO . . . . . . . . . . .  	NUMBER	0006	
READ . . . . . . . . . . . . . .  	NUMBER	003F	
READ_SECTOR  . . . . . . . . . .  	NUMBER	0000	
READ_WRITE . . . . . . . . . . .  	NUMBER	0008	
REDIRECTOR . . . . . . . . . . .  	NUMBER	0000	
REGFLG . . . . . . . . . . . . .  	L BYTE	051A	DATA	Global
REGMEM . . . . . . . . . . . . .  	L BYTE	0481	DATA	Global
REGSAVE  . . . . . . . . . . . .  	L WORD	046D	DATA	Global
REGTABLEN  . . . . . . . . . . .  	NUMBER	000E	
rel_high_sec . . . . . . . . . .  	L WORD	0002	DATA	Global
rel_low_sec  . . . . . . . . . .  	L WORD	0000	DATA	Global
rel_read_write_tab . . . . . . .  	L DWORD	0000	DATA	Global
rel_rw_add . . . . . . . . . . .  	L DWORD	0006	DATA	Global
rel_sec_num  . . . . . . . . . .  	L WORD	0004	DATA	Global
RENAME . . . . . . . . . . . . .  	NUMBER	0056	
RESERVED_BITS_MASK . . . . . . .  	NUMBER	FE00	
RMDIR  . . . . . . . . . . . . .  	NUMBER	003A	

SAVESTATE  . . . . . . . . . . .  	L 	0437	DATA	Global
SEGDIF . . . . . . . . . . . . .  	NUMBER	0000	
SEGFLG . . . . . . . . . . . . .  	L BYTE	051D	DATA	Global
SEGSAVE  . . . . . . . . . . . .  	L WORD	046F	DATA	Global
SERVERCALL . . . . . . . . . . .  	NUMBER	005D	
SETBLOCK . . . . . . . . . . . .  	NUMBER	004A	
SETCNTC  . . . . . . . . . . . .  	ALIAS	 TRUE		
SETDPB . . . . . . . . . . . . .  	NUMBER	0053	
SET_CTRL_C_TRAPPING  . . . . . .  	NUMBER	0033	
Microsoft (R) Macro Assembler Version 5.10                  2/14/25 23:44:19
DEBDATA.SAL - PC DOS                                        Symbols-12


SET_CURRENT_PDB  . . . . . . . .  	NUMBER	0050	
SET_DATE . . . . . . . . . . . .  	NUMBER	002B	
SET_DEFAULT_DRIVE  . . . . . . .  	NUMBER	000E	
SET_DMA  . . . . . . . . . . . .  	NUMBER	001A	
SET_DRIVEID_OPTION . . . . . . .  	NUMBER	0001	
SET_INTERRUPT_VECTOR . . . . . .  	NUMBER	0025	
SET_OEM_HANDLER  . . . . . . . .  	NUMBER	00F8	
SET_PRINTER_FLAG . . . . . . . .  	NUMBER	0064	
SET_TIME . . . . . . . . . . . .  	NUMBER	002D	
SET_VERIFY_ON_WRITE  . . . . . .  	NUMBER	002E	
SF_BUSY  . . . . . . . . . . . .  	NUMBER	-0001	
SF_CLOSE_NODATE  . . . . . . . .  	NUMBER	4000	
SF_DEFAULT_NUMBER  . . . . . . .  	NUMBER	0005	
SF_FSDA  . . . . . . . . . . . .  	BYTE	0019	
SF_ISFCB . . . . . . . . . . . .  	NUMBER	8000	
SF_ISNET . . . . . . . . . . . .  	NUMBER	8000	
SF_LRU . . . . . . . . . . . . .  	WORD	0015	
SF_NETID . . . . . . . . . . . .  	BYTE	0019	
SF_NET_SPOOL . . . . . . . . . .  	NUMBER	0800	
SF_NO_INHERIT  . . . . . . . . .  	NUMBER	1000	
SF_OPENAGE . . . . . . . . . . .  	WORD	0017	
SF_PIPE  . . . . . . . . . . . .  	NUMBER	2000	
SF_SERIAL_ID . . . . . . . . . .  	WORD	000B	
SHAREF . . . . . . . . . . . . .  	NUMBER	0000	
SHARING_COMPAT . . . . . . . . .  	NUMBER	0000	
SHARING_DENY_BOTH  . . . . . . .  	NUMBER	0010	
SHARING_DENY_NONE  . . . . . . .  	NUMBER	0040	
SHARING_DENY_READ  . . . . . . .  	NUMBER	0030	
SHARING_DENY_WRITE . . . . . . .  	NUMBER	0020	
SHARING_MASK . . . . . . . . . .  	NUMBER	00F0	
SHARING_NET_FCB  . . . . . . . .  	NUMBER	0070	
SHARING_NO_INHERIT . . . . . . .  	NUMBER	0080	
SIFLG  . . . . . . . . . . . . .  	L BYTE	0514	DATA	Global
SINGLE_QUOTE . . . . . . . . . .  	NUMBER	0027	
SIREG  . . . . . . . . . . . . .  	NUMBER	4953	
SSINTSAV . . . . . . . . . . . .  	L DWORD	042E	DATA	Global
STDAUX . . . . . . . . . . . . .  	NUMBER	0003	
STDERR . . . . . . . . . . . . .  	NUMBER	0002	
STDIN  . . . . . . . . . . . . .  	NUMBER	0000	
STDOUT . . . . . . . . . . . . .  	NUMBER	0001	
STDPRN . . . . . . . . . . . . .  	NUMBER	0004	
STD_AUX_INPUT  . . . . . . . . .  	NUMBER	0003	
STD_AUX_OUTPUT . . . . . . . . .  	NUMBER	0004	
STD_CON_INPUT  . . . . . . . . .  	NUMBER	0001	
STD_CON_INPUT_FLUSH  . . . . . .  	NUMBER	000C	
STD_CON_INPUT_NO_ECHO  . . . . .  	NUMBER	0008	
STD_CON_INPUT_STATUS . . . . . .  	NUMBER	000B	
STD_CON_OUTPUT . . . . . . . . .  	NUMBER	0002	
STD_CON_STRING_INPUT . . . . . .  	NUMBER	000A	
STD_CON_STRING_OUTPUT  . . . . .  	NUMBER	0009	
STD_PRINTER_OUTPUT . . . . . . .  	NUMBER	0005	
SWITCHAR . . . . . . . . . . . .  	L BYTE	044F	DATA	Global
SYSVER . . . . . . . . . . . . .  	ALIAS	 FALSE		

TCOUNT . . . . . . . . . . . . .  	L WORD	0488	DATA	Global
TEMP . . . . . . . . . . . . . .  	L BYTE	0477	DATA	Global	Length = 0004
TEMPLEN  . . . . . . . . . . . .  	NUMBER	0086	
TRANSADD . . . . . . . . . . . .  	L DWORD	0454	DATA	Global
TRUE . . . . . . . . . . . . . .  	NUMBER	FFFF	
TRUEBYTE . . . . . . . . . . . .  	NUMBER	00FF	
TSTFLG . . . . . . . . . . . . .  	L BYTE	051C	DATA	Global

UNLINK . . . . . . . . . . . . .  	NUMBER	0041	
UPPER_A  . . . . . . . . . . . .  	NUMBER	0041	
UPPER_C  . . . . . . . . . . . .  	NUMBER	0043	
UPPER_E  . . . . . . . . . . . .  	NUMBER	0045	
UPPER_F  . . . . . . . . . . . .  	NUMBER	0046	
UPPER_L  . . . . . . . . . . . .  	NUMBER	004C	
UPPER_M  . . . . . . . . . . . .  	NUMBER	004D	
UPPER_N  . . . . . . . . . . . .  	NUMBER	004E	
UPPER_P  . . . . . . . . . . . .  	NUMBER	0050	
UPPER_S  . . . . . . . . . . . .  	NUMBER	0053	
UPPER_X  . . . . . . . . . . . .  	NUMBER	0058	
UPPER_Z  . . . . . . . . . . . .  	NUMBER	005A	
USEROPER . . . . . . . . . . . .  	NUMBER	005E	

Microsoft (R) Macro Assembler Version 5.10                  2/14/25 23:44:19
DEBDATA.SAL - PC DOS                                        Symbols-13


VEC_BREAKPOINT . . . . . . . . .  	NUMBER	0003	
VEC_CRIT_ERR . . . . . . . . . .  	NUMBER	0024	
VEC_CTRL_BREAK . . . . . . . . .  	NUMBER	0023	
VEC_PRIMITIVE_DISK_READ  . . . .  	NUMBER	0025	
VEC_PRIMITIVE_DISK_WRITE . . . .  	NUMBER	0026	
VEC_SING_STEP  . . . . . . . . .  	NUMBER	0001	
VEC_TERM_ADDR  . . . . . . . . .  	NUMBER	0022	

WAITPROCESS  . . . . . . . . . .  	NUMBER	004D	
WRITE  . . . . . . . . . . . . .  	NUMBER	0040	
WRITE_SECTOR . . . . . . . . . .  	NUMBER	0000	

XDUP . . . . . . . . . . . . . .  	NUMBER	0045	
XDUP2  . . . . . . . . . . . . .  	NUMBER	0046	
xm_alloc_pg  . . . . . . . . . .  	L WORD	041B	DATA	Global
xm_deall_han . . . . . . . . . .  	L WORD	0011	DATA	Global
XM_ERR80 . . . . . . . . . . . .  	NUMBER	0080	
XM_ERR83 . . . . . . . . . . . .  	NUMBER	0083	
XM_ERR84 . . . . . . . . . . . .  	NUMBER	0084	
XM_ERR85 . . . . . . . . . . . .  	NUMBER	0085	
XM_ERR86 . . . . . . . . . . . .  	NUMBER	0086	
XM_ERR87 . . . . . . . . . . . .  	NUMBER	0087	
XM_ERR88 . . . . . . . . . . . .  	NUMBER	0088	
XM_ERR89 . . . . . . . . . . . .  	NUMBER	0089	
XM_ERR8A . . . . . . . . . . . .  	NUMBER	008A	
XM_ERR8B . . . . . . . . . . . .  	NUMBER	008B	
XM_ERR8D . . . . . . . . . . . .  	NUMBER	008D	
XM_ERR8E . . . . . . . . . . . .  	NUMBER	008E	
XM_ERR8F . . . . . . . . . . . .  	NUMBER	008F	
xm_frame . . . . . . . . . . . .  	L WORD	0419	DATA	Global
xm_handle  . . . . . . . . . . .  	L WORD	0013	DATA	Global
xm_handle_pages_buf  . . . . . .  	L BYTE	0019	DATA	Global	Length = 0400
xm_handle_ret  . . . . . . . . .  	L WORD	0015	DATA	Global
xm_han_alloc . . . . . . . . . .  	L WORD	0421	DATA	Global
xm_han_total . . . . . . . . . .  	L WORD	041F	DATA	Global
xm_log . . . . . . . . . . . . .  	L BYTE	000F	DATA	Global
XM_NOT_INST  . . . . . . . . . .  	NUMBER	00FF	
xm_page  . . . . . . . . . . . .  	L BYTE	000E	DATA	Global
xm_page_cnt  . . . . . . . . . .  	L WORD	0017	DATA	Global
xm_phy . . . . . . . . . . . . .  	L BYTE	0010	DATA	Global
xm_total_pg  . . . . . . . . . .  	L WORD	041D	DATA	Global
XNAMETRANS . . . . . . . . . . .  	NUMBER	0060	
XNXCMD . . . . . . . . . . . . .  	L BYTE	044E	DATA	Global
XNXOPT . . . . . . . . . . . . .  	L BYTE	044D	DATA	Global

?PLM . . . . . . . . . . . . . .  	NUMBER	0000	
?WIN . . . . . . . . . . . . . .  	NUMBER	0000	
@CPU . . . . . . . . . . . . . .  	TEXT  0101h		
@FILENAME  . . . . . . . . . . .  	TEXT  debdata		
@VERSION . . . . . . . . . . . .  	TEXT  510		


   2837 Source  Lines
   2949 Total   Lines
    942 Symbols

  43174 + 173804 Bytes symbol space free

      0 Warning Errors
      0 Severe  Errors
